:1000000000800010CD000000B91C0000BB1C0000E7
:10001000BD1C0000BF1C0000C11C0000000000004F
:10002000000000000000000000000000C31C0000F1
:10003000C51C000000000000C71C0000C91C000017
:10004000CB1C0000CB1C0000CB1C0000CB1C000014
:10005000CB1C0000CB1C0000CB1C0000CB1C000004
:10006000CB1C0000CB1C0000CB1C0000CB1C0000F4
:10007000CB1C0000CB1C0000CB1C0000CB1C0000E4
:10008000CB1C0000CB1C0000CB1C0000CB1C0000D4
:10009000CB1C0000CB1C0000CB1C0000CB1C0000C4
:1000A000BD170000CB1C0000CB1C0000CB1C0000C7
:1000B000CB1C0000CB1C0000CB1C0000CB1C0000A4
:1000C000CB1C0000CB1C0000CB1C0000014880476B
:1000D00001480047E91E0000A521000040F210037E
:1000E000C1F200031A780AB901201870704700BFE6
:1000F00040F20000C1F2000008B503682BB140F2E5
:100100000003C0F2000303B1984708BD4CF240035E
:10011000C2F209035B6903F48063002B07D140F24C
:100120001103C1F200034FF001021A7006E040F221
:100130001103C1F200034FF000021A70704700BFB4
:1001400082B04CF24003C2F209034FF0FF02DA61C1
:100150004CF22003C2F209034FF07042DA6140F220
:100160001203C1F200031B7803F001038DF807307E
:100170009DF80730002B0CD14CF26003C2F209034A
:100180004CF26002C2F20902D26942F08062DA6186
:100190000BE04CF26003C2F209034CF26002C2F2BF
:1001A0000902926942F080629A6140F21203C1F240
:1001B00000031B7803F002038DF807309DF8073029
:1001C000002B0CD14CF24003C2F209034CF2400266
:1001D000C2F20902D26942F02002DA610BE04CF26D
:1001E0004003C2F209034CF24002C2F209029269D2
:1001F00042F020029A6140F21203C1F200031B7820
:1002000003F004038DF807309DF80730002B0CD164
:100210004CF24003C2F209034CF24002C2F209025E
:10022000D26942F01002DA610BE04CF24003C2F2F4
:1002300009034CF24002C2F20902926942F0100234
:100240009A6140F21203C1F200031B7803F0080325
:100250008DF807309DF80730002B0CD14CF240038D
:10026000C2F209034CF24002C2F20902D26942F022
:100270000802DA610BE04CF24003C2F209034CF2CF
:100280004002C2F20902926942F008029A6140F209
:100290001203C1F200031B7803F010038DF807303E
:1002A0009DF80730002B0CD14CF24003C2F2090339
:1002B0004CF24002C2F20902D26942F00402DA6151
:1002C0000BE04CF24003C2F209034CF24002C2F2CE
:1002D0000902926942F004029A6140F21203C1F2EB
:1002E00000031B7803F020038DF807309DF80730DA
:1002F000002B0CD14CF22003C2F209034CF2200275
:10030000C2F20902D26942F00042DA610BE04CF21B
:100310002003C2F209034CF22002C2F209029269E0
:1003200042F000429A6140F21203C1F200031B78CE
:1003300003F040038DF807309DF80730002B0CD1F7
:100340004CF22003C2F209034CF22002C2F209026D
:10035000D26942F00052DA610BE04CF22003C2F2A3
:1003600009034CF22002C2F20902926942F00052E3
:100370009A6140F21203C1F200031B7823F07F035D
:100380008DF807309DF80730002B0CD14CF220037C
:10039000C2F209034CF22002C2F20902D26942F011
:1003A0008052DA610BE04CF22003C2F209034CF2F6
:1003B0002002C2F20902926942F080529A6102B0B0
:1003C000704700BF08B54CF24003C2F209034FF07A
:1003D000FF021A604CF22003C2F209034FF0704290
:1003E0001A604CF26003C2F209034FF080621A6097
:1003F00000F0E6FC4FF0010000F05AFDFEE700BF00
:1004000082B001900091FEE708B540F23403C1F2DA
:100410000003DB78022B10D0032B11D0012B12D15B
:10042000FFF774FE40F21103C1F200031A7840F2A4
:100430001C03C1F200031A7005E04FF0000304E052
:100440004FF0000301E04FF00103184608BD00BF64
:1004500008B540F23403C1F20003DB78022B06D06A
:10046000032B11D0012B12D14FF0000311E040F209
:100470001C03C1F200031A7840F21203C1F2000318
:100480001A70FFF75DFE02E04FF0000301E04FF04D
:100490000103184608BD00BF40F23403C1F2000357
:1004A0009B781A4640F21403C1F200039A5C40F2B2
:1004B0001C03C1F200031A704FF001031846704785
:1004C00040F23403C1F200039B781A4640F2340331
:1004D000C1F20003D97840F21403C1F20003995429
:1004E0004FF001031846704740F21503C1F20003B4
:1004F0001A7840F21C03C1F200031A704FF0010396
:100500001846704740F23403C1F200039A7840F273
:100510001503C1F200031A704FF00103184670472B
:1005200040F24803C1F200034FF000021A8040F28B
:100530002803C1F200034FF000021A7040F23003AA
:10054000C1F200034FF000021A7040F22403C1F21E
:1005500000034FF001121A6040F22C03C1F20003B5
:100560004FF000021A60704708B54FF0000040F2EB
:100570003401C1F2000100F07FFE08BD00B583B078
:1005800040F24003C1F200039B88082B03D94FF0CF
:100590000803019305E040F24003C1F200039B8889
:1005A000019340F24003C1F200031B684FF080004A
:1005B0001946019A00F0C6FE0346019340F240033B
:1005C000C1F200031A68019B1A4440F24003C1F2D1
:1005D00000031A6040F24003C1F200039A88019BB5
:1005E0009BB2C3EB02039AB240F24003C1F2000394
:1005F0009A8003B000BD00BF00B583B040F2400355
:10060000C1F200031B684FF00000194600F034FEF1
:100610000346019340F24003C1F200031A68019BB4
:100620001A4440F24003C1F200031A6040F2400352
:10063000C1F200039A88019B9BB2C3EB02039AB2FA
:1006400040F24003C1F200039A8003B000BD00BF36
:1006500008B54FF080004FF000014FF0000200F0AD
:1006600071FE08BD08B54FF0000040F21C01C1F258
:10067000000100F001FE08BD00B585B040F2340372
:10068000C1F200031B78C3F30403DBB2002B02D0DA
:10069000012B70D0AFE040F23403C1F20003DB78ED
:1006A000022B10D0032B4AD0012B60D140F2400323
:1006B000C1F2000342F23422C0F200021A604FF08D
:1006C0001203029356E042F24823C0F20003019362
:1006D0004FF00003039312E0019B1B78002B0AD01C
:1006E000019B9A78DB784FEA032343EA02039BB22B
:1006F000019A13440193039B03F10103039340F216
:100700003403C1F200039B781A46039B9A42E3D15B
:10071000019B1B78002B02D14FF0000382E040F2D6
:100720004003C1F20003019A1A60019B9A78DB78BA
:100730004FEA032343EA02039BB202931AE040F21A
:100740003403C1F200039B781A4642F26C23C0F2D4
:1007500000031A4440F24003C1F200031A6040F261
:100760004003C1F200031B681B78029302E04FF0C4
:10077000000357E042E040F23403C1F20003DB78AB
:10078000222B17D0232B2FD0212B30D140F2340332
:10079000C1F200031B79002B02D04FF0000341E0AF
:1007A00040F24003C1F20003204A1A604FF00903EF
:1007B00002931FE040F23403C1F200031B79002BC7
:1007C00002D04FF000032DE040F24003C1F20003DD
:1007D00042F20422C0F200021A6042F23023C0F258
:1007E00000031B88029305E04FF000031AE04FF06E
:1007F000000317E002E04FF0000313E040F2400373
:10080000C1F200039B881A46029B9A4206D9029BBA
:100810009AB240F24003C1F200039A80FFF7AEFEA5
:100820004FF00103184605B000BD00BF5A2200007A
:1008300000B585B040F23403C1F200039B78002B71
:1008400059D042F24823C0F2000300934EE0009BCF
:100850005B78042B2BD0052B2DD0022B3DD1009B98
:100860005A7940F23403C1F200039B789A420ED1C8
:1008700040F23403C1F200039A7840F23003C1F22F
:1008800000031A704FF0010000F014FC25E0009BFB
:100890000393009B9A78DB784FEA032343EA020331
:1008A0009BB2039A13440393039B00931EE0009BA7
:1008B000DB78019311E0019B002B0ED1009B9B780C
:1008C00003F08F030293009B184600F023FC02986C
:1008D00000F06AFC029800F091FC009B0393009BDF
:1008E0001B78039A13440393039B0093009B1B788C
:1008F000002BACD10AE040F23003C1F200034FF00C
:1009000000021A704FF0000000F0D4FB40F23403F4
:10091000C1F200039A7840F23003C1F200031B7861
:100920009A4202D14FF0010301E04FF00003184654
:1009300005B000BD00B583B00190019B03F1FF330A
:10094000062B00F2928101A252F823F069090000FF
:100950005F0B00001F0C00006B0C00006B0C000014
:100960004F0C0000450C0000FFF7FEFD40F2340381
:10097000C1F20003DA8840F24003C1F200039A801A
:1009800040F23403C1F200031B78C3F34113DBB21E
:10099000012B55D0022B00F0D480002B40F0D280E8
:1009A00040F23403C1F200035B78062B24D0092BFC
:1009B00025D0052B00D042E040F23403C1F2000301
:1009C0001B78C3F30403DBB2002B00D013E040F22A
:1009D0003403C1F200039A7840F22803C1F2000305
:1009E0001A70FFF735FE40F22803C1F200031B78AE
:1009F000184600F04BFB22E0FFF73EFE1FE040F2FE
:100A00003403C1F200031B78C3F30403DBB2002BF1
:100A100000D014E0FFF70CFF0346002B0BD14FF082
:100A2000800000F0FFFB40F24003C1F200034FF0F2
:100A300000029A8003E0FFF70BFE01F0B7F88DE0AB
:100A400040F23403C1F200031B78C3F30403DBB2AA
:100A5000012B00D074E040F23403C1F200031B7993
:100A6000002B6DD140F23403C1F200035B7803F137
:100A7000FF330A2B64D801A252F823F0A90A000020
:100A8000DF0A0000110B0000410B0000410B0000C9
:100A9000410B0000410B0000410B0000CB0A00009D
:100AA000010B0000330B0000FFF7AEFC0346002BE8
:100AB0000AD040F24003C1F2000340F21C02C1F22E
:100AC00000021A60FFF75AFD3AE040F24003C1F21B
:100AD000000340F21C02C1F200021A6030E0FFF78E
:100AE000DBFC0346002B0AD040F24003C1F20003B6
:100AF00040F21C02C1F200021A60FFF73FFD1FE046
:100B0000FFF7DEFC0346002B01D0FFF7A1FD17E045
:100B1000FFF7EAFC0346002B0AD040F24003C1F283
:100B2000000340F21C02C1F200021A60FFF726FD2A
:100B300006E0FFF7E7FC0346002B01D0FFF788FD36
:100B40000CE00BE04FF0800000F06CFB40F2400343
:100B5000C1F200034FF000029A8086E085E040F287
:100B60003403C1F200031B7803F08003002B73D120
:100B700040F24003C1F200039B88002B6ED0FFF7C8
:100B80003BFD40F24003C1F200039B88002B67D17C
:100B900040F23403C1F200031B78C3F34113DBB20C
:100BA000002B02D0012B05D032E04FF0800000F086
:100BB00039FB31E040F23403C1F200031B78C3F388
:100BC0000403DBB2012B02D0022B16D01AE040F254
:100BD0003403C1F200031B79002B09D1FFF738FC65
:100BE0000346002B03D14FF0800000F01BFB0EE00A
:100BF0004FF0800000F016FB09E04FF0800000F09D
:100C000011FB04E04FF0800000F00CFB04E003E077
:100C10004FF0800000F006FBFFF71AFD25E040F2E0
:100C20003403C1F200031B7803F08003002B19D0BA
:100C300040F24003C1F200039B88002B14D0FFF761
:100C40009DFC12E04FF0800000F002FB0DE04FF041
:100C5000000000F0FDFA08E000BF06E000BF04E07D
:100C600000BF02E000BF00E000BF03B000BD00BF56
:100C700082B003468DF807304EF20013CEF2000327
:100C80009DF907204FEA52129DF8071001F01F014D
:100C90004FF0010000FA01F143F8221002B0704752
:100CA00084B00190019B03F00F034FEA43030393C9
:100CB000019B03F08003002B03D0039B03F101038E
:100CC0000393039B184604B0704700BF82B00190A5
:100CD0004CF20003C5F200034FF01002C3F80822E3
:100CE0004CF20003C5F20003019AC3F810224CF243
:100CF0000003C5F20003D3F8003203F01003002B09
:100D0000F5D002B0704700BF82B0019000914CF264
:100D10000003C5F200034FF01002C3F808224CF2A2
:100D20000003C5F20003019AC3F810224CF200033D
:100D3000C5F20003D3F8003203F01003002BF5D006
:100D40004CF20003C5F200034FF01002C3F8082272
:100D50004CF20003C5F20003009AC3F810224CF2D3
:100D60000003C5F20003D3F8003203F01003002B98
:100D7000F5D002B0704700BF82B001904CF2000382
:100D8000C5F200034FF03002C3F808224CF2000312
:100D9000C5F20003019AC3F810224CF20003C5F219
:100DA0000003D3F8003203F02003002BF5D04CF2FF
:100DB0000003C5F20003D3F81432184602B070479E
:100DC00008B54CF20003C4F202034CF20002C4F274
:100DD0000202526822F070525A604CF20003C4F2D0
:100DE00002034CF20002C4F20202526842F0A05226
:100DF0005A604CF20003C4F202034CF20002C4F247
:100E00000202D26822F0405222F03002DA604CF244
:100E10000003C4F202034CF20002C4F20202D268E0
:100E200042F0005242F01002DA604CF20003C4F2C9
:100E300002034CF20002C4F20202126922F44022C0
:100E40001A614CF20003C4F202034CF20002C4F235
:100E50000202126942F480221A614CF20003C4F2C9
:100E60000F034CF20002C4F20F02D2F8C42042F089
:100E70000042C3F8C4204CF20003C5F200034FF057
:100E80001A02C3F8F42F4CF20003C5F20003D3F8A2
:100E9000F83F03F01A031A2BF5D14FF01800FFF7B3
:100EA000E7FE00F01BF84FF0000000F0EFF808BD7F
:100EB00000B583B00190019B002B04D040F20013D9
:100EC000C0F2010301E04FF4807340F20050C0F221
:100ED000FE001946FFF718FF03B000BD82B04CF2C8
:100EE0000003C5F200034FF00002C3F848224CF2A1
:100EF0000003C5F200034FF00802C3F84C224CF285
:100F00000003C5F200034FF00102C3F848224CF27F
:100F10000003C5F200034FF00802C3F84C224CF264
:100F20000003C5F20003D3F8003203F48073002BF2
:100F3000F5D04CF20003C5F200034FF0FF32C3F8C6
:100F400038224CF20003C5F200034FF0FF32C3F821
:100F500034224CF20003C5F200034FF0FF32C3F815
:100F600008224CF20003C5F200034FF00C02C3F854
:100F700004224CF20003C5F2000340F20002C2F268
:100F80000802C3F880224CF20003C5F200034FF0C0
:100F9000FF32C3F854224CF20003C5F200034FF0B5
:100FA000FF32C3F88C224CF20003C5F200034FF06D
:100FB0000002C3F888224CF20003C5F200034FF090
:100FC000FF32C3F8A4224CF20003C5F200034FF035
:100FD000FF32C3F8B0224CF20003C5F200034FF019
:100FE000FF32C3F8BC224CF20003C5F200034FF0FD
:100FF0000702C3F8942240F2CC03C1F200034FF081
:1010000000021A6040F2CC03C1F200034FF000026C
:101010005A604FF00003019315E0019A40F24C032F
:10102000C1F200034FF0000143F82210019A40F290
:101030000003C2F208034FF0000143F82210019BA5
:1010400003F101030193019B1F2BE6D902B0704706
:10105000704700BF704700BF08B540F24803C1F2B7
:1010600000031B8803F00203002B09D040F200505C
:10107000C0F2FE0040F20011C0F20101FFF744FE91
:1010800008BD00BF82B0019002B0704700B583B0C8
:101090000190019B43F080034FEA034343F48073C4
:1010A00040F20050C0F2D0001946FFF72DFE03B009
:1010B00000BD00BF00B583B00190019B002B04D0A0
:1010C00040F20013C0F2010301E04FF4807340F2DC
:1010D0000050C0F2D8001946FFF716FE4CF200038C
:1010E000C5F200034FF00302C3F844224CF20003A0
:1010F000C5F20003D3F8003203F48073002BF5D05F
:101100004CF20003C5F200034FF48072C3F80822CA
:1011100003B000BD00B585B00190019B9B781846D7
:10112000FFF7BEFD034603934CF20003C5F2000334
:101130004CF20002C5F20002D2F84412039A4FF0BA
:10114000010000FA02F241EA0202C3F844224CF222
:101150000003C5F20003039AC3F848224CF20003CF
:10116000C5F20003019A117952794FEA022242EA4C
:10117000010292B2C3F84C224CF20003C5F2000304
:10118000D3F8003203F48073002BF5D04CF2000347
:10119000C5F200034FF48072C3F8082205B000BD09
:1011A00082B0019002B0704700B583B00190019801
:1011B000FFF776FD03464FEA034343F4800343F40D
:1011C000A06318464FF48071FFF79EFD03B000BD89
:1011D00000B583B001900198FFF762FD03464FEA26
:1011E000034343F4800343F4A063184640F2001124
:1011F000C0F22001FFF788FD03B000BD00B583B049
:1012000001900198FFF74CFD03464FEA034343F476
:10121000800343F4A06318464FF48071FFF774FD18
:1012200003B000BD00B583B001900198FFF738FD11
:1012300003464FEA034343F4800343F4A063184694
:1012400040F20011C0F20101FFF75EFD03B000BDE6
:1012500000B583B001900198FFF722FD03464FEAE5
:10126000034343F4800343F4A06318464FF48071B2
:10127000FFF74AFD03B000BD00B585B001900091B5
:101280004CF20003C5F20003019A02F00F024FEA8C
:10129000820242F00102C3F828224CF20003C5F298
:1012A0000003D3F820320293029B03F40063002B67
:1012B000F3D0029B4FEA83534FEA935302934FF0CC
:1012C000000303930FE0009A4CF20003C5F2000301
:1012D000D3F818321360009B03F104030093039BBF
:1012E00003F101030393029B03F103034FEA93020B
:1012F000039B9A42E7D84CF20003C5F200034FF07B
:101300000002C3F82822019B41F2482242FA03F36B
:1013100003F00103002B10D10198FFF7C1FC034635
:101320004FEA034343F4A0631846FFF7CFFC40F2B3
:101330000050C0F2F200FFF7C9FC029B184605B04E
:1013400000BD00BF00B587B00390029101924CF23E
:101350000003C5F20003039A02F00F024FEA820273
:1013600042F00202C3F828224CF20003C5F2000347
:10137000019AC3F824224FF0000305930FE04CF2CA
:101380000003C5F20003029A1268C3F81C22029BF4
:1013900003F104030293059B03F101030593019BF1
:1013A00003F103034FEA9302059B9A42E7D84CF2FC
:1013B0000003C5F200034FF00002C3F8282203988F
:1013C000FFF76EFC03464FEA034343F4A06318465D
:1013D000FFF77CFC40F20050C0F2FA00FFF776FC09
:1013E000019B184607B000BD00B589B0019000917F
:1013F000009B1B7BC3F34003DBB205930198FFF70F
:101400004FFC034602934FF000030393029A40F20D
:101410004C03C1F2000353F82230049335E0049BDF
:101420000393009B1B7B03F00103002B2AD1059A39
:1014300042F2D023C0F2000353F82230039AC3EBE8
:101440000202059942F2D823C0F2000353F821307A
:10145000B2FBF3F30693059A059940F2CC03C1F26F
:10146000000353F82110069B4FF0010000FA03F32C
:101470006FEA030301EA030140F2CC03C1F2000367
:1014800043F82210039B1B680493049B002BC6D1D6
:101490004FF00003069313E0059A40F2CC03C1F22B
:1014A000000353F82220069B4FF0010101FA03F3D9
:1014B00002EA0303002B07D0069B03F10103069306
:1014C000069B1F2BE8D900E000BF069B202B02D112
:1014D0004FF0000396E0059A059940F2CC03C1F263
:1014E000000353F82110069B4FF0010000FA03F3AC
:1014F00041EA030140F2CC03C1F2000343F8221099
:10150000059A42F2D023C0F2000353F82220059935
:1015100042F2D823C0F2000353F82130069901FBB0
:1015200003F313440493039B002B13D0009B1B7BFA
:1015300003F00103002B0DD0039B049A1A60039B58
:1015400003F10403039A02F10402126842F0040258
:101550001A600FE0029A40F24C03C1F200030499B2
:1015600043F82210029A40F20003C2F208030499E1
:1015700043F82210049B0793079B4FF000021A6068
:10158000079B03F104030793009B1B7BC3F38003BA
:10159000DBB21A46009B1B7BC3F34003DBB24FEA6E
:1015A000031342EA0302009BDB884FEA431342EA3B
:1015B0000302009B9B884FEA034342EA03031A4657
:1015C000079B1A60079B03F104030793009B1A68AB
:1015D000079B1A60079B03F104030793009B5B7B47
:1015E0004FEA03231A46079B1A60079B03F1040383
:1015F0000793059B002B03D0009B9A68079B1A60FA
:101600004FF00103184609B000BD00BF10B582B00D
:1016100001904CF20004C5F200040198FFF740FB72
:1016200003464FF0010202FA03F3C4F8883202B015
:1016300010BD00BF10B582B001904CF20004C5F29D
:1016400000040198FFF72CFB03464FF0010202FA59
:1016500003F3C4F88C3202B010BD00BF00B585B0F2
:1016600001900198FFF71CFB024640F20003C2F212
:10167000080353F822300293029B002B02D14FF053
:10168000000337E0029B03F10C031B680393039BE9
:101690004FEA530303F00F03092B29D801A252F894
:1016A00023F000BFCD160000D3160000D9160000AD
:1016B000DF160000F1160000F1160000F116000020
:1016C000F1160000E5160000EB1600004FF00103D4
:1016D00010E04FF002030DE04FF003030AE04FF07B
:1016E000050307E04FF0040304E04FF0060301E0B8
:1016F0004FF6FF73184605B000BD00BF00B585B0BA
:1017000001900198FFF7CCFA024640F20003C2F2C2
:10171000080353F822300293029B002B02D14FF0B2
:10172000FF3305E0029B03F108031B680393039B4F
:10173000184605B000BD00BF00B585B00190019806
:10174000FFF7AEFA024640F20003C2F2080353F874
:1017500022300293029B002B02D14FF0FF3307E0AF
:10176000029B03F10C031B680393039B4FEA134393
:10177000184605B000BD00BF00B583B040F2005070
:10178000C0F2F500FFF7A2FA40F20020C0F2F50027
:10179000FFF7F2FA0346019340F20020C0F2F50091
:1017A000FFF7EAFA03464FEA0323019A42EA0303EA
:1017B0000193019B184603B000BD00BF00B585B082
:1017C0004CF20003C5F20003D3F8003200934CF250
:1017D0000003C5F20003009AC3F80822009B03F03F
:1017E0000803002B27D040F20050C0F2FE00FFF7A4
:1017F0006DFA40F20020C0F2FE00FFF7BDFA03468A
:101800000193019B03F01003002B03D0FFF766FB4D
:1018100000F0C8F9019B03F00803002B00F0BF8122
:10182000019B03F00403002B02D0FFF711FCB7E18A
:10183000FFF710FCB4E1009B03F00403002B00F061
:101840008C8081E04FF0000302937AE04CF20003B9
:10185000C5F20003D3F83022029B4FF0010101FAD8
:1018600003F302EA0303002B67D0029B4FEA530302
:1018700003934CF20003C5F20003029A4FF00101FA
:1018800001FA02F2C3F838224CF20003C5F2000359
:10189000D3F8003203F02003002BF5D04CF2000304
:1018A000C5F20003D3F814320193029B03F0010345
:1018B000002B2BD1029B002B14D1019B03F00403BE
:1018C000002B0FD042F2E023C0F200031B68002B74
:1018D00008D042F2E023C0F200031B684FF0010081
:1018E00098472AE0039A42F2E023C0F2000353F83B
:1018F0002230002B20D0039A42F2E023C0F20003F2
:1019000053F822304FF00200984716E0039B002B5B
:1019100003D14FF00300FFF70DF8039B012B03D118
:101920004FF0030000F058F9039B022B05D14FF054
:10193000030000F065F900E000BF029B03F1010322
:101940000293029B1F2B81D94CF20003C5F20003C6
:10195000D3F83032002B7FF475AF4CF20003C5F2A0
:101960000003D3F8903203F00103DBB2002B55D013
:101970004CF20003C5F20003D3F8A03201934FF0FC
:101980000203029340E0029B4FF0010202FA03F3CC
:101990001A46019B02EA0303002B31D0029B4FEA57
:1019A00053030393029B03F00103002B13D1039A0B
:1019B00042F2E023C0F2000353F82230002B1ED085
:1019C000039A42F2E023C0F2000353F822304FF0B2
:1019D0000800984714E0039A42F2E023C0F20003A3
:1019E00053F82230002B0BD0039A42F2E023C0F2CE
:1019F000000353F822304FF00900984700E000BF81
:101A0000029B03F101030293029B1F2BBBD94CF2F3
:101A10000003C5F20003019AC3F8A4224CF20003AC
:101A2000C5F20003D3F8903203F00203002B55D027
:101A30004CF20003C5F20003D3F8AC3201934FF02F
:101A40000203029340E0029B4FF0010202FA03F30B
:101A50001A46019B02EA0303002B31D0029B4FEA96
:101A600053030393029B03F00103002B13D1039A4A
:101A700042F2E023C0F2000353F82230002B1ED0C4
:101A8000039A42F2E023C0F2000353F822304FF0F1
:101A90000A00984714E0039A42F2E023C0F20003E0
:101AA00053F82230002B0BD0039A42F2E023C0F20D
:101AB000000353F822304FF00B00984700E000BFBE
:101AC000029B03F101030293029B1F2BBBD94CF233
:101AD0000003C5F20003019AC3F8B0224CF20003E0
:101AE000C5F20003D3F8903203F00403002B57D063
:101AF0004CF20003C5F20003D3F8B83201934FF063
:101B00000203029340E0029B4FF0010202FA03F34A
:101B10001A46019B02EA0303002B31D0029B4FEAD5
:101B200053030393029B03F00103002B13D1039A89
:101B300042F2E023C0F2000353F82230002B1ED003
:101B4000039A42F2E023C0F2000353F822304FF030
:101B50000C00984714E0039A42F2E023C0F200031D
:101B600053F82230002B0BD0039A42F2E023C0F24C
:101B7000000353F822304FF00D00984700E000BFFB
:101B8000029B03F101030293029B1F2BBBD94CF272
:101B90000003C5F20003019AC3F8BC2200E000BFB5
:101BA00005B000BD08B5FEF7BBFC08BD08B540F2A6
:101BB0003003C1F200031B78002B0BD0FEF7A6FA0E
:101BC0004FF0810040F21101C1F200014FF001021B
:101BD000FFF7B8FB08BD00BF00B583B00190019BC3
:101BE000032B0BD1FEF792FA4FF0810040F2110166
:101BF000C1F200014FF00102FFF7A4FB03B000BDEA
:101C000000B583B00190019B032B0BD1FEF77EFA48
:101C10004FF0820040F21101C1F200014FF00102C9
:101C2000FFF790FB03B000BD00B583B00190019BAE
:101C3000032B0BD1FEF76AFA4FF0830040F211013B
:101C4000C1F200014FF00102FFF77CFB03B000BDC1
:101C500082B0019002B0704782B0019002B070472C
:101C600082B0019002B0704782B0019002B070471C
:101C700082B0019002B0704782B0019002B070470C
:101C800082B0019002B0704782B0019002B07047FC
:101C900082B0019002B0704782B0019002B07047EC
:101CA00082B0019002B0704782B0019002B07047DC
:101CB00082B001900091FEE7FEE7FEE7FEE7FEE757
:101CC000FEE7FEE7FEE7FEE7FEE7FEE74CF2000375
:101CD000C4F20F03D3F888304FEA136303F0030311
:101CE000032B40F0AA804CF20003C4F20F03D3F898
:101CF0000C3103F00303032B00F2F48001A252F82D
:101D000023F000BF151D0000791D0000DF1D00003D
:101D1000151D00004CF20003C4F20F03D3F8883005
:101D20004FEA43434FEA534303F1010241F20023D8
:101D3000C0F27A0303FB02F24CF20003C4F20F0379
:101D4000D3F888304FEA134303F0FF0303F1010394
:101D5000B2FBF3F24CF20003C4F20F03D3F80431E8
:101D600003F0FF0303F10103B2FBF3F240F20803B7
:101D7000C1F200031A60B6E04CF20003C4F20F0394
:101D8000D3F888304FEA43434FEA534303F101024B
:101D900043F20063C0F26E1303FB02F24CF2000345
:101DA000C4F20F03D3F888304FEA134303F0FF0364
:101DB00003F10103B2FBF3F24CF20003C4F20F0390
:101DC000D3F8043103F0FF0303F10103B2FBF3F294
:101DD00040F20803C1F200031A6000BF83E04CF236
:101DE0000003C4F20F03D3F888304FEA43434FEAAD
:101DF000534303F101034FEA03424CF20003C4F2E0
:101E00000F03D3F888304FEA134303F0FF0303F1C5
:101E10000103B2FBF3F24CF20003C4F20F03D3F858
:101E2000043103F0FF0303F10103B2FBF3F240F2CC
:101E30000803C1F200031A6055E04CF20003C4F23B
:101E40000F03D3F80C3103F00303032B4BD801A28B
:101E500052F823F0651E0000911E0000BD1E000018
:101E6000651E00004CF20003C4F20F03D3F80431E6
:101E700003F0FF0303F1010240F60013C0F23D033B
:101E8000B3FBF2F240F20803C1F200031A602AE049
:101E90004CF20003C4F20F03D3F8043103F0FF0344
:101EA00003F1010241F60033C0F2B703B3FBF2F2D3
:101EB00040F20803C1F200031A6014E04CF2000380
:101EC000C4F20F03D3F8043103F0FF0303F101035D
:101ED0004FF40042B2FBF3F240F20803C1F20003F8
:101EE0001A6000E000BF70474CF20003C4F20F0319
:101EF0004FF02002C3F8A0214CF20003C4F20F03FC
:101F0000D3F8A03103F02003002B09D04CF20003DA
:101F1000C4F20F03D3F8A03103F04003002BF5D037
:101F20004CF20003C4F20F034FF00302C3F8042184
:101F30004CF20003C4F20F034FF00002C3F8A821D3
:101F40004CF20003C4F20F034FF00002C3F8AC21BF
:101F50004CF20003C4F20F034FF00102C3F80C214E
:101F60004CF20003C4F20F0340F26302C0F2050218
:101F7000C3F884204CF20003C4F20F034FF0AA020E
:101F8000C3F88C204CF20003C4F20F034FF055024B
:101F9000C3F88C204CF20003C4F20F034FF001028F
:101FA000C3F880204CF20003C4F20F034FF0AA02E2
:101FB000C3F88C204CF20003C4F20F034FF055021B
:101FC000C3F88C204CF20003C4F20F03D3F888301E
:101FD00003F08063002BF5D04CF20003C4F20F0332
:101FE0004FF00302C3F880204CF20003C4F20F0349
:101FF0004FF0AA02C3F88C204CF20003C4F20F0386
:102000004FF05502C3F88C204CF20003C4F20F03CA
:10201000D3F8883003F04073002BF5D04CF2000366
:10202000C4F20F034FF02302C3F8A4204CF20003C4
:10203000C4F20F034FF0AA02C3F8AC204CF2000325
:10204000C4F20F034FF05502C3F8AC204CF200036A
:10205000C4F20F034FF00102C3F8A0204CF20003BA
:10206000C4F20F034FF0AA02C3F8AC204CF20003F5
:10207000C4F20F034FF05502C3F8AC204CF200033A
:10208000C4F20F03D3F8A83003F48063002BF5D01B
:102090004CF20003C4F20F034FF00302C3F8A02078
:1020A0004CF20003C4F20F034FF0AA02C3F8AC20B5
:1020B0004CF20003C4F20F034FF05502C3F8AC20FA
:1020C0004CF20003C4F20F03D3F8A83003F44073BA
:1020D000002BF5D04CF20003C4F20F0348F2DE727D
:1020E000C0F22842C3F8C4204CF20003C4F20F032C
:1020F0004FF00002C3F8C8214CF20003C4F20F03F2
:1021000043F23A021A604EF60053CEF200034FF04B
:1021100000029A60704700BF08B500F04BF807480E
:1021200000B10068064901B109680022FEF74AF9CA
:10213000044B0BB1AFF30080FEE700BF00000000CE
:10214000000000000000000080B51448144B21E09E
:102150005C689968DD688C420CD0002205E0A61806
:102160000832D6E9008941E902898C460831AA4241
:10217000F5D101E004EB050C1C696146002204E086
:1021800008320026002741E902670831A242F7D150
:10219000143301380028DBD1FFF7BEFF0100000037
:1021A0004023000001498D46014908470080001086
:1021B0004921000070B542F22C3642F22C35C0F2B3
:1021C0000006C0F20005761BB61006D0002455F8B4
:1021D000243001349847A642F9D842F22C3542F215
:1021E0003036C0F20005C0F20006761B00F098F809
:1021F000B61006D0002455F8243001349847A64282
:10220000F9D870BD0600FF0901A1010509190129CE
:10221000031500250195037501810295017505815E
:10222000010508094B15002501950875019102C0AB
:102230002C000000120100020000000851C201221F
:102240000001042042010000090222000101008077
:102250003209040000010300005C092100010001B3
:10226000222C000705810304002000000403090458
:102270001C034E00580050002000530045004D0044
:10228000490043004F004E004400200022034C0050
:1022900050004300310037007800780020004800EB
:1022A00049004400200020002000200020001A03E4
:1022B000440045004D004F00300030003000300039
:1022C000300030003000300008034800490044006E
:1022D0008000082080010820100000001400000089
:1022E00035090000D91B0000011C0000000000009F
:1022F00000000000000000000000000000000000DE
:1023000000000000000000000000000000000000CD
:1023100000000000000000000000000000000000BD
:10232000F8B500BFF8BC08BC9E467047F10000003D
:10233000F8B500BFF8BC08BC9E467047DD00000041
:1023400000000000602300000000001010000000EA
:04235000C8000000C1
:0823540078DDFF7F01000000AD
:10236000000000000000000000E1F5050000000092
:00000001FF
